S01900006F70656E626C745F73746D3332663330332E7372656303
S315080000000030002025050008F5040008F70400085C
S31508000010F9040008FB040008FD04000800000000BD
S31508000020000000000000000000000000FF040008B7
S315080000300105000800000000030500080505000882
S31508000040750500087505000875050008750500089A
S31508000050750500087505000875050008750500088A
S31508000060750500087505000875050008750500087A
S31508000070750500087505000875050008750500086A
S31508000080750500087505000875050008750500085A
S31508000090750500087505000875050008750500084A
S315080000A0750500087505000875050008750500083A
S315080000B075050008750500080000000075050008AC
S315080000C0750500080000000000000000750500081E
S315080000D0000000007505000875050008750500088C
S315080000E075050008750500080000000000000000FE
S315080000F000000000000000000000000000000000F2
S3150800010000000000000000000000000000000000E1
S3150800011000000000000000007505000875050008CD
S3150800012000000000000000000000000000000000C1
S3150800013000000000000000000000000000000000B1
S31508000140750500087505000800000000000000009D
S315080001500000000000000000000000000000000091
S315080001600000000000000000000000000000000081
S315080001700000000000000000000000000000000071
S30D080001800000000075050008E7
S3150800018810B5054C237833B9044B13B10448AFF3BB
S3150800019800800123237010BD100000200000000015
S315080001A8381D000808B5034B1BB103490348AFF3CC
S315080001B8008008BD0000000014000020381D000853
S315080001C801F0DABB01F0E7BB08B54FF090431869B0
S315080001D810F4007002D000F02FF8012008BD642042
S315080001E800F002B800F006B8014B1880704700BF47
S315080001F82C00002010B50C4C01F06EFB22689042CA
S315080002080DD30A4B0A4A1878082148B901201870EC
S31508000218916101F061FB074B1B881844206010BDEB
S31508000228002018709162F4E7300000202E000020A4
S31508000238000400482C000020014B08229A627047E7
S3150800024800040048054B5A6902435A615B6982B043
S3150800025818400190019B02B0704700BF0010024089
S3150800026808B5264B1A6822F0070242F002021A60FD
S315080002781A6802F00702022AFAD1214B1A6842F0D4
S3150800028801021A601A689107FCD51A6822F0F80262
S3150800029842F080021A605A6822F4741242F4601214
S315080002A85A60DA6A22F00F02DA621A6842F0807235
S315080002B81A601A689201FCD55A6822F0F0025A6048
S315080002C85A6822F4E06242F480625A605A6822F454
S315080002D860525A605A6822F0030242F002025A60D3
S315080002E85A6802F00C02082AFAD1064800F0D8FF24
S315080002F80020BDE8084000F04DB900BF00200240C4
S31508000308001002400090D00380B58EB000F066F960
S31508000318FFF7A6FF1822002107A801F001FD364DB0
S315080003284FF40030FFF78EFF08274FF4802000248B
S31508000338FFF788FF01264FF40073AF6207A94FF04D
S315080003489040CDE907340B9600F0DEFD07A928464C
S31508000358CDE909440B94CDE9077600F0D5FD1C22B2
S3150800036821460DEB020001F0DBFC2146182201A804
S3150800037801F0D6FC214BDA6942F40032DA61DB690E
S3150800038803F4003300934FF40030009BFFF75AFF3D
S3150800039848F204020223CDE901230323CDE90334F5
S315080003A801A907234FF090400594069300F0ACFD89
S315080003B84FF41643CDE907340C23CDE90B34CDE9C0
S315080003C809440D940E4C07A9204600F00FFFA368B0
S315080003D823F48063A360636823F490436360A36887
S315080003E823F02A03A360236833432360FFF7E8FE54
S315080003F8FFF7E8FEFCE700BF0004004800100240CB
S31508000408004400400A4B9A6942F001029A619A69C7
S3150800041882B002F001020092009ADA6942F080522C
S31508000428DA61DB6903F080530193019B02B07047D8
S315080004380010024010B5044688B01422002103A80B
S3150800044801F06EFC2268134B9A4221D103F5D63384
S315080004580321DA6942F00072DA61DA6902F0007299
S315080004680192019A5A6942F400325A615B6903F4A7
S3150800047800330293029B4FF4C0520223CDE90323AB
S315080004880923CDE906134FF0904003A900F026FC8E
S3150800049808B010BD0064004008B500F0D5FD114845
S315080004A80823836200F0DAFC4FF0904000F0D6FC8F
S315080004B80D4BDA6922F00072DA61DA6922F4003241
S315080004C8DA615A6922F480225A615A6922F400329A
S315080004D85A61DA6922F08052DA619A6922F00102D1
S315080004E89A6108BD00040048001002407047FEE7FC
S315080004F8FEE7FEE7FEE770477047704700F080B8EA
S31508000508054BD3F8882042F47002C3F888204FF0C8
S3150800051800629A60704700BF00ED00E0DFF834D04B
S31508000528002103E00C4B5B58435004310B480C4B35
S3150800053842189A42F6D30B4A02E0002342F8043BD3
S31508000548094B9A42F9D3FFF7DBFF01F0C5FBFFF722
S31508000558DBFEFEE7003000201C1E00080000002015
S31508000568100000201000002070050020FEE700009B
S3150800057810B5074B4FF0FF3200241A611C61DA6088
S31508000588DC609A629C62FFF787FF204610BD00BFB1
S315080005980010024038B50E4A0E4B054618784FF437
S315080005A87A73B3FBF0F31068B0FBF3F000F060FA67
S315080005B8044658B90F2D09D8024629464FF0FF3088
S315080005C800F022FA044B20461D6038BD0120FCE7DE
S315080005D8000000200400002008000020074A08B58B
S315080005E8136843F010031360032000F0FBF900209A
S315080005F8FFF7D0FFFFF706FF002008BD00200240DE
S31508000608034A044B11681B780B441360704700BFF4
S31508000618480500200400002038B5044600286ED096
S3150800062890F820300BB9FFF705FF2268136823F006
S315080006380203136001F058F9054623685A689107BA
S3150800064851D41A6842F001021A6001F04DF90546BC
S3150800065823685A68D20754D5227E012A1A680CBF1D
S3150800066842F0800222F080021A60627E012A1A6825
S315080006780CBF42F0400222F040021A60A27E012A0C
S315080006881A680CBF42F0200222F020021A60E27EA5
S31508000698012A1A680CBF22F0100242F010021A60EA
S315080006A8227F012A1A680CBF42F0080222F00802C3
S315080006B81A60627F012A1A680CBF42F0040222F007
S315080006C804021A60D4E902210A4321690A436169C6
S315080006D80A43616801390A43DA6100200123606226
S315080006E884F8203038BD01F0FFF8401B0A28A4D941
S315080006F8636A43F400336362052384F820300120D3
S31508000708F0E701F0F1F8401B0A28A1D9F0E790F8BC
S315080007182030013B012B70B55FD80368D3F8002257
S3150800072842F00102C3F800224A69D3F81C52012490
S3150800073802F01F0004FA00F0C4432540C3F81C520F
S31508000748CD6985BBD3F80C52CE682540C3F80C5240
S315080007588D8803EBC20245EA0645C2F840528E6800
S315080007680D8845EA0645C2F844528A696ABBD3F831
S3150800077804222240C3F804220A6952BBD3F8142279
S315080007882240C3F814220A6A012A02BFD3F81C2297
S315080007981043C3F81C02D3F8002222F00102C3F85A
S315080007A80022002070BD012DDFD1D3F80C520E6847
S315080007B80543C3F80C528D8803EBC20245EA064581
S315080007C8C2F840528E688D89CBE7D3F804220243D3
S315080007D8D0E7D3F814220243D3E7436A43F48023C5
S315080007E843620120DEE738B590F82030012B04462D
S315080007F81FD10268022380F82030136823F001030A
S31508000808136001F071F805462368586810F001006E
S3150800081801D1606238BD01F067F8401B0A28F3D990
S31508000828636A43F400336362052384F820300120A1
S31508000838F0E7436A43F400234362F8E7F0B590F813
S3150800084820500668013D012DB46840D814F0E05FD1
S3150800085839D0C4F30164032C4FF0010505D1436A66
S3150800086843F400034362012027E0A5401D60D1E94F
S31508000878020704F1180308BB086847EA40501B0139
S315080008882401F05033190869097DC3F88401012940
S3150800089802BFD3F8841141F48071C3F88411344433
S315080008A85168C4F88C111268C4F88821D3F88021D5
S315080008B842F00102C3F880210020F0BD4D68384394
S315080008C840EAC500DBE7436A43F40013CAE7436A0C
S315080008D843F48023C6E790F82030013B012B08D85B
S315080008E803689B68890631EA030314BF01200020C0
S315080008F8704700207047F0B590F82040013C012C5D
S315080009086BD8066841B9F468A40707D1436A43F463
S3150800091800134362012055E03469F5E70C013519DF
S31508000928D5F8B07107F004079760002F4BD1D5F8B2
S31508000938B0717F0D1760D5F8B07107F00207D76058
S31508000948D5F8B47107F00F071761D5F8B471D5F85B
S31508000958B4512644C7F307272D0C97615561D6F875
S31508000968B8211A7002682244D2F8B821120A5A70B5
S3150800097802682244D2F8B821120C9A7002682244F6
S31508000988D2F8B821120EDA7002682244D2F8BC21CD
S315080009981A7102682244D2F8BC21120A5A710268EE
S315080009A82244D2F8BC21120C9A7102681444D4F86D
S315080009B8BC21120EDA71036851B9DA6842F02002CE
S315080009C8DA600020F0BDD5F8B071FF085760B2E7C5
S315080009D81A6942F020021A61F3E7436A43F480234E
S315080009E897E70000074AD36823F4E0631B041B0C47
S315080009F843F0BF63000243F4003300F4E0600343A6
S31508000A08D360704700ED00E0174B70B5DC68C4F397
S31508000A180224C4F10705042D04F1040328BF04259C
S31508000A284FF0FF36062B06FA05F38CBF033C002465
S31508000A3821EA0303A34006FA04F422EA0404002878
S31508000A4843EA0403A8BF00F160404FEA0313BCBF9A
S31508000A5800F00F00054ADBB2AABF00F5614013543F
S31508000A6880F8003370BD00BF00ED00E014ED00E02B
S31508000A780138B0F1807F0AD2064B074A5860F02140
S31508000A8882F823100020072298601A607047012010
S31508000A98704700BF10E000E000ED00E00B4AD3689D
S31508000AA813F0100305D00A49CB6943F00203CB615A
S31508000AB81023D268520706D50549CA6942F00102C9
S31508000AC8CA6143F00403014AD36070470020024014
S31508000AD850050020064B186910F0800007D0054A13
S31508000AE85A6002F188325A601869C0F3C010704714
S31508000AF80020024023016745034A136943F080032F
S31508000B0813610020704700BF00200240F8B505466B
S31508000B1800F0EAFE104C07462646E368D9070FD4C4
S31508000B28E3689A0644BF2023E360F368DB0603D428
S31508000B38F06810F0040007D0FFF7B0FF012003E0C3
S31508000B48681CEAD00DB90320F8BD00F0CDFEC01B1D
S31508000B58A842E2D9F7E700BF002002402DE9F84F7E
S31508000B68244C1E46237E012B05460F4690463FD049
S31508000B7801234CF250302376FFF7C8FFA0BB012D9E
S31508000B8803D0022D0CBF022504254FF00009DFF813
S31508000B9868A0CB464FEA0913C3F12001A3F1200246
S31508000BA806FA01F128FA03F3C4F81CB00B4326FA2F
S31508000BB802F21343DAF810209BB242F00102CAF88F
S31508000BC810204CF2503027F81930FFF79FFFDAF853
S31508000BD8103023F00103CAF8103028B909F10109C1
S31508000BE85FFA89F39D42D5D800232376BDE8F88FA6
S31508000BF80220FBE75005002000200240064B002291
S31508000C08DA61064B1A6942F004021A611A6942F057
S31508000C1840021A61704700BF5005002000200240B4
S31508000C28064B0022DA61064B1A6942F002021A617B
S31508000C3858611A6942F040021A6170475005002047
S31508000C48002002402DE9F041224D2B7E012B074654
S31508000C5888463DD003680124A3422C764CF25030CE
S31508000C6813D1FFF753FF20B1012000232B76BDE8E7
S31508000C78F081FFF7C3FF4CF25030FFF747FF164ADB
S31508000C88136923F004031361EFE7FFF73FFF002812
S31508000C98EAD14FF0FF33C8F8003020467E680E4C7C
S31508000CA8D7E9013203EBC223B342DED93046FFF750
S31508000CB8B7FF4CF25030FFF729FF236923F00203E8
S31508000CC8236110B1C8F80060CFE706F50066E7E7C4
S31508000CD80220CCE750050020002002402DE9F04FFD
S31508000CE885B00B68DFF870E1594A01934FF00F0990
S31508000CF80023019CDC4002D105B0BDE8F08F012431
S31508000D0804FA03F8019C18EA040500F098804C6870
S31508000D1824F0100A4FEA430C03260AF1FF3706FAAD
S31508000D280CF6012F6FEA060611D8876807EA060B3C
S31508000D38CF6807FA0CF747EA0B078760476827EA78
S31508000D480808C4F300179F4047EA08074760C768BA
S31508000D5807EA06088F6807FA0CF747EA0807BAF198
S31508000D68020FC76014D14FEAD30800EB880803F0CE
S31508000D78070AD8F820704FEA8A0A09FA0AFB27EA06
S31508000D880B0B0F6907FA0AF747EA0B07C8F820702A
S31508000D9807683E4004F0030707FA0CFC4CEA060607
S31508000DA80660E6004BD5DEF8186046F00106CEF870
S31508000DB81860DEF8186023F0030707F1804706F085
S31508000DC8010607F58037039603F0030C039EBE68F1
S31508000DD84FEA8C0C09FA0CF8B0F1904F26EA080885
S31508000DE82FD01C4EB0422ED006F58066B0422CD0C5
S31508000DF806F58066B04214BF0526032606FA0CF6E1
S31508000E0846EA0806BE601668EF4314F4803F0CBF2E
S31508000E183E402E431660566814F4003F0CBF3E4009
S31508000E282E435660966814F4801F0CBF3E402E4326
S31508000E389660D668A40254BF3E402E43D660013356
S31508000E4857E70026DAE70126D8E70226D6E700BFDD
S31508000E58000401400004004800100240B0F1904F19
S31508000E680AD1244B9A6A42F400329A629A6A22F4A0
S31508000E7800329A62002070471F4B98420BD103F143
S31508000E88784303F503339A6A42F480229A629A6A87
S31508000E9822F48022EDE7194B98420BD103F17843E7
S31508000EA803F502339A6A42F400229A629A6A22F48D
S31508000EB80022DEE7124B98420BD103F1784303F57B
S31508000EC801339A6A42F480129A629A6A22F4801264
S31508000ED8CFE70C4B98420BD103F1784303F5FE3361
S31508000EE89A6A42F480029A629A6A22F48002C0E7F1
S31508000EF80120704700100240000400480008004816
S31508000F08000C0048001400482DE9F04F02460D6809
S31508000F1895FAA5F44FF0010EB4FA84F403264FF0B7
S31508000F280F0C6FEA050835FA04F001D1BDE8F08F11
S31508000F380EFA04F32B406CD04868471E012F1ED8BA
S31508000F48976893FAA3F9B9FA89F993FAA3FA4FEACB
S31508000F58490906FA09F927EA0909BAFA8AFA8F68D5
S31508000F684FEA4A0A07FA0AF749EA070797605768E5
S31508000F7808EA0709CF686F4349EA07075760D76839
S31508000F8893FAA3F9B9FA89F993FAA3FA4FEA490938
S31508000F9806FA09F927EA0909BAFA8AFA0F694FEA2D
S31508000FA84A0A07FA0AF749EA07070228D7601DD145
S31508000FB893FAA3F7B7FA87F7072FD1F814A02ADC0C
S31508000FC8D2F820B093FAA3F7B7FA87F793FAA3F9F2
S31508000FD8B9FA89F9BF000CFA07F74FEA89092BEA23
S31508000FE807070AFA09FA47EA0A071762D2F80090C1
S31508000FF893FAA3F7B7FA87F793FAA3F3B3FA83F33F
S315080010087F0006FA07F75B0029EA070798400743AF
S315080010181760013487E7D2F824B04FEA132999FAFA
S31508001028A9F7B7FA87F799FAA9F9B9FA89F9BF00B2
S315080010380CFA07F74FEA89092BEA07070AFA09FAA1
S3150800104847EA0A075762D1E71E4B1A6842F00102B7
S3150800105882B01A601A689207FCD51A6822F0F80254
S3150800106842F080021A604FF0FF3201920199164A3F
S315080010780A400192019A5A605A6812F00C0FFBD17D
S315080010881A680192019A22F0847222F48032019237
S31508001098019A1A60186810F00070FBD11A6822F4D1
S315080010A880221A604FF41F025860D86218630192AA
S315080010B8019A9A6098605A6A42F080725A6202B037
S315080010C8704700BF001002400CC0FFF8034B044AE3
S315080010D85B68C3F30313D35CD8407047001002401B
S315080010E8501D0008034B044A5B68C3F30223D35C0C
S315080010F8D840704700100240601D0008034B044A98
S315080011085B68C3F3C223D35CD8407047001002401B
S31508001118601D00080D4B0E495A680E4802F48032C5
S31508001128002A08BF0846D96A5B684FF4701292FA13
S31508001138A2F2B2FA82F203F47013D340023301F032
S315080011480F010131B0FBF1F0584370470010024017
S3150800115800093D0000127A00044B5B6803F00C0393
S31508001168082B01D1FFF7D6BF014870470010024087
S3150800117800127A0010B50446FFF7EEFF2060FFF765
S31508001188A5FF6060FFF7AEFFA0606068FFF7B6FFCF
S31508001198E06010BD08B518BB124A136B03F00303C9
S315080011A8022B0ED0032B05D0012B11D1BDE8084020
S315080011B8FFF7D2BF136813F0020F0B4B18BF184678
S315080011C808BD136A13F0020F18BF4FF40040F7E77B
S315080011D8FFF7C2FFFFF77AFFBDE80840FFF782BFAF
S315080011E80020EDE70010024000127A0030B50446E8
S315080011F8006810F0010085B00D4602D0012005B040
S3150800120830BDEA686B68216813432A691343AA69DB
S3150800121813431F4A0A40134323606368AA6823F4E2
S31508001228405313436360A3686A6923F440731343FE
S31508001238A360184B9C4219D1FFF7ACFF0028DDD0F4
S315080012482A68002ADAD0A969B1F5004F4FEA52038D
S3150800125818D103EB4003B3FBF2F34FF6F0721A40CA
S31508001268C3F342031343E3600020C8E70A4B9C42D2
S3150800127804D16846FFF77EFF0298DFE7074B9C42D2
S31508001288BCD1F6E70344B3FBF2F39BB2EBE700BF26
S31508001298F369FFEF00380140004400400048004069
S315080012A8014B1860704700BF0000002072B67047EF
S315080012B862B67047F0B58BB06846FFF75BFF2A4DF4
S315080012C8029C00210E464FF4FA774FF47A73B4FB62
S315080012D8F3F46B184A5D5B78D01800FB0770B4FB0B
S315080012E8F0FC00FB1C4028B91FFA8CF6701EB0F5F6
S315080012F8806F08D302312429EBD1AF211B4800F0AF
S31508001308FBFA00231A461A4C1A492160013A013B8E
S315080013180025012712041B052046226163612576EC
S315080013286576A576E77625776577C4E90255666012
S31508001338FFF772F94CF6E0434FF6E072CDE900354F
S315080013480423CDE9022369460E2320460993CDE9ED
S315080013580555079704950897FFF7D9F92046FFF723
S3150800136842FA0BB0F0BD00BFA41D0008681D0008AE
S31508001378340000200064004030B589B040F2E173BB
S3150800138802930023CDE904330691024601AB02A96C
S315080013980A48FFF753FA78B900F09EFA074C00F1A5
S315080013A8320501992046FFF796FA28B100F065FB41
S315080013B800F092FAA842F4D909B030BD34000020EA
S315080013C810B588B00C46034601AA00210848FFF75D
S315080013D892FA58B9019A40F267639A4204D1039B74
S315080013E813B9059B2370012008B010BD0020FBE740
S315080013F834000020FFF75ABF10B500F0A1F9C8B1AC
S31508001408FEF7E2FEB0B100F007FBFFF7B1F800F00F
S315080014183BFA00F097F9084B20F0604020F07F006F
S31508001428986000F08FF94468FFF742FF2346BDE845
S315080014381040184710BD00BF00ED00E0F8B5144687
S31508001448461A4FF6FF75013CA4B2AC4200D1F8BD66
S315080014580B788B554F1C00F010FB3946F3E72DE93E
S31508001468F8430546FFF736FB002405F104082F68FC
S3150800147858F8046004EB070900F0FFFA324600231F
S3150800148849460220FFF76AFB60B9E359B3420BD114
S315080014980434B4F5007FEAD10124FFF72DFB204672
S315080014A8BDE8F8830024F8E70446F6E738B50E4B96
S315080014B8984204460D4607D00C4A914212D0FFF7C7
S315080014C8CEFF10B904460BE0094C23689D4207D0A5
S315080014D820464FF4007240F8045B2946FFF7AEFF32
S315080014E8204638BD1C46F0E76002002000200008A8
S315080014F85C0000202DE9F0419846036821F4FF7640
S31508001508013304460D46174626F0010606D140F86B
S31508001518046B4FF400723146FFF790FF2368B34215
S3150800152805D020463146FFF7C1FF0446E8B12368CF
S315080015380435ED1A254406F50076B84400F09DFAF8
S31508001548231DEB1AB3F5007F06D320463146FFF76D
S31508001558ADFF044648B1051D17F8013B05F8013BE0
S315080015684745EBD10120BDE8F0810020FBE70000E4
S31508001578034A4FF0FF331360024A1360704700BFEF
S315080015885C0000206002002030B40E4C4D1E0B464D
S31508001598211A8D4213D80C49884210D9411E19447C
S315080015A8A1420CD820F4FF71084C21F00101A14290
S315080015B8014630BC0CBF06480648FFF79BBF00200B
S315080015C830BC7047FFFF0008FF1F0008002000080E
S315080015D8600200205C00002030B51D4D85B04A1E0B
S315080015E82B1A00249A42009420D820F4FF63194A3B
S315080015F823F00703934219D9421E0A44AA4215D86A
S315080016080144C91AC1F3CF25C1F30A0109B1013545
S31508001618ADB20024CDE9014301230393FFF75AFA33
S31508001628A3B2AB4205D30124FFF766FA204605B0F4
S3150800163830BD00F022FA694601A8FFF703FB01341A
S3150800164820B9029B03F500630293E9E70024EBE758
S31508001658FFFF0008FF1F000807B50F4A1368013384
S3150800166817D0D2E901310B44D1680C480B441169EB
S315080016780B4451690B449169D2690B44134402AA75
S315080016885B4242F8043D0421FFF77EFF03B05DF88C
S3150800169804FB0120FAE700BF600200208821000841
S315080016A80D4B0E4A1B68126813440D4A12681344F8
S315080016B80C4A126813440C4A126813440B4A1268F7
S315080016C813440B4A126813440A4A1268D3420CBFD9
S315080016D801200020704700BF0020000804200008E9
S315080016E8082000080C20000810200008142000080C
S315080016F818200008882100080A4808B50368013335
S3150800170805D109480368013306D1012008BDFFF74A
S31508001718A6FE0028F5D1F9E7FFF7A1FE003018BFA5
S315080017280120F3E7600200205C00002000487047AB
S3150800173800200008FFF71CBFFFF726BFFFF74CBFBE
S31508001748FFF7AEBFFFF7F2BF08B5FFF785FF18B179
S31508001758BDE80840FFF7D0BF08BD000038B5084CFB
S31508001768208500F0B9F800F10A05E3691B0605D4D7
S3150800177800F083F900F0B0F8A842F6D938BD00BFE2
S315080017880044004010B50D4C236823F0010388B0C7
S3150800179823604FF461420023CDE9012301A90C22F5
S315080017A82046CDE90333CDE905230793FFF71EFD48
S315080017B8236843F00103236008B010BD00440040C5
S315080017C8402970B506460C4603D96F21094800F02A
S315080017D893F82046FFF7C2FF3546A4B2AB1B9BB267
S315080017E89C4200D870BD00F048F915F8010BFFF7C0
S315080017F8B5FFF3E7C81D0008F8B51E4D1E4A2C7834
S315080018080E46ACB9D3699B0602D400242046F8BD17
S31508001818938C1A4ADBB21370013B3F2BF5D800F0BC
S315080018285BF8174B1860174B1C7001232B70EDE7F4
S31508001838D46914F0200414D0124C10492378978CD4
S31508001848CA18013357700A78DBB29A422370DCD17A
S315080018580131FFF7F3FD00232B7023783370012439
S31508001868D4E700F039F8064B1B6864339842CCD99C
S315080018782C70CBE7A504002000440040640400202F
S31508001888A8040020A6040020024B00221A605A6009
S315080018989A60704710E000E008B5FFF7F5FF054BBA
S315080018A84FF6FF125A60052100229A601960024B0A
S315080018B81A6008BD10E000E0AC040020044B1B6861
S315080018C8DB0341BF034A136801331360704700BF3F
S315080018D810E000E0AC04002008B5FFF7EFFF014B65
S315080018E8186808BDAC04002008B5FFF7E7FF014BE8
S315080018F8186808BDAC04002008B500F0BEF8FCE777
S3150800190810B500F0B1F8012814D00B4C2378012B38
S3150800191810D1FFF7E1FF094B094A1B6812681344FF
S3150800192803F5FA73984205D300232370BDE81040DF
S31508001938FFF762BD10BD00BFB4040020B004002044
S31508001948B804002008B5044B1B78012B03D1FFF710
S31508001958C3FF024B186008BDB4040020B804002071
S3150800196808B5044B01221A70FFF7ECFFBDE80840DA
S31508001978FFF7C6BFB404002008B5FFF73BFD00F023
S315080019887AF8FFF789FFFFF7D5FE00F00FF8BDE8EC
S315080019980840FFF7E5BF08B500F06FF8FFF78EFFB8
S315080019A800F014F8BDE80840FFF7AABF10B5064CC2
S315080019B800F070F8FFF77EFC01232370FFF7E2FEBC
S315080019C80023237010BD00BF0C00002007B510487F
S315080019D80DF10701FFF7F4FC012806D10D4B9DF818
S315080019E8071018700A4800F071F80DF10701084841
S315080019F8FFF702FF012807D1064B9DF80710044890
S31508001A0800221A7000F062F803B05DF804FB00BF04
S31508001A18BC0400200C0000207047000070B5094C73
S31508001A282278012A06460D4602D1C9B2FFF7A4FC58
S31508001A3823781BB9E9B23046FFF7C2FEBDE8704005
S31508001A4800F03CB80C000020044B1B78013BDBB2C5
S31508001A58022B9ABF024AD05C402070470C0000202F
S31508001A68061E0008FFF7F0BF08B500F01FF800309B
S31508001A7818BF012008BDFEF7B2BBFEF7B3BB0000CE
S31508001A88034BFE22DA7002221871A3F84420704725
S31508001A98FC040020044B00229A6483F84320A3F828
S31508001AA844201A809A707047FC040020024B187864
S31508001AB8003018BF01207047FC040020024B0022A2
S31508001AC883F84320704700BFFC040020F8B5037864
S31508001AD87E4CFF2B05462CD1E37010230125237174
S31508001AE8002363712580FFF7AFFFA071FFF7BAFFE0
S31508001AF8E071FFF7B7FF0823000A20726572A5721E
S31508001B08A4F84430FFF716FE94F84330012B02D1A7
S31508001B181020FFF7B5FFB4F94410002940F3D48024
S31508001B28012384F8433089B26948BDE8F840FFF7CD
S31508001B3875BF2678012E40F0C780F32B58D01FD8DA
S31508001B48CF2B00F0BE8007D8C92B00F08380CC2B9A
S31508001B5800F08980202030E0D12B00F0AB80C0F05F
S31508001B688C80D22BF6D10025FF23E3702571657189
S31508001B78FFF76AFFE571A0712572657207232BE0E6
S31508001B88FA2B4CD00BD8F52B11D028D3F62BE1D14C
S31508001B98FF23E3704368A364A4F84460B4E7FD2B05
S31508001BA849D0FE2B51D0FC2BD4D1002005E0FFF7F5
S31508001BB84BFF6A78904203D82220FFF761FFA3E714
S31508001BC8A16C201DFFF73AFCFF23E3706A78A36C23
S31508001BD81344A3646B780133A4F8443094E7FFF7F9
S31508001BE833FF6B788342E7D26968A1646A78E8E7C5
S31508001BF8FF23E370A66C476800253744BE4207D121
S31508001C080123A3800023C4F80750A3710823E3E738
S31508001C1816F8013B1D44EDB2FFF72FFFEEE7FF2349
S31508001C28E3702C4BA364002323716371A371072304
S31508001C38C4F80730EAE7FF23E37062786271002385
S31508001C482371E38023720623C6E700232380FF2334
S31508001C58E370A1E7A76CFFF7F7FE6A1C411E384632
S31508001C68FFF76AFD08B93120A7E7FF23E370FFF7F6
S31508001C78EBFEA36C013803448DE7FFF7E5FE6B78A6
S31508001C880138984298DDFF23E370A4F84460697820
S31508001C9829B9FFF759FD00287FF436AFE3E7AA1CF0
S31508001CA8A06CFFF749FD0028DDD06A78A36C1344B9
S31508001CB8A36429E74168A06CFFF740FD0028C6D150
S31508001CC8D1E7FFF799FBC2E7F8BD00BFFC0400207F
S31508001CD8FF040020091E000870B50D4E0D4CA41B04
S31508001CE8A4100025A54209D10B4E0C4C00F020F88B
S31508001CF8A41BA4100025A54205D170BD56F82530A9
S31508001D0898470135EEE756F8253098470135F2E742
S31508001D18141E0008141E0008141E0008181E0008C1
S31508001D2802440346934200D1704703F8011BF9E7BA
S31508001D38F8B500BFF8BC08BC9E467047F8B500BFA2
S30D08001D48F8BC08BC9E46704772
S31508001D50000000000000000001020304060708094D
S31508001D600000000001020304433A2F576F726B2FDD
S31508001D70736F6674776172652F4F70656E424C5447
S31508001D802F5461726765742F536F757263652F419F
S31508001D90524D434D345F53544D333246332F6361AE
S31508001DA06E2E6300050206020603070308030903ED
S31508001DB009040A040B040C040C050D050E050F0591
S31508001DC00F06100610071008433A2F576F726B2F2D
S31508001DD0736F6674776172652F4F70656E424C54E7
S31508001DE02F5461726765742F536F757263652F413F
S31508001DF0524D434D345F53544D333246332F72732D
S31508001E003233322E63000800004F70656E424C5420
S30908001E1000000000C0
S30908001E14AD01000806
S30908001E188901000826
S31508001E1C00127A0001000000100000000400000007
S70508000525C8
